:100000004AC072C071C070C06FC06FC06DC06CC09C
:100010006BC06AC069C068C067C066C065C00000C8
:1000200000000000000000000000000000000000D0
:1000300000000000000000000000000000000000C0
:1000400000002167B1FF030405070A0E1319212BD5
:10005000364353657990AAC6E6FFFFFFFFFFFFFF17
:10006000FFFFFFFFFFFFFFFFFFFFFFFFFF0000009D
:100070000000000000000000000000000000000080
:10008000000008121C2834414E5C6B7C8FA3B8CF53
:10009000E6FFFFFFFF0011241FBECFE5D2E0DEBF69
:1000A000CDBF20E0A0E6B0E001C01D92A238B207AB
:1000B000E1F7E1E6F0E085E5808781E08383148263
:1000C000128286831182ACE6B0E08EEF15968C9397
:1000D00015978DEF17968C9388E081878FE4828740
:1000E000612C712C7ED0BCC08BCF189525B7277E94
:1000F00025BF29B7226029BF21E022BF019728F040
:1001000020E188952150E9F7F9CF089588EE93E032
:10011000EDCF81EA87B986EC86B9369A0895369A8A
:100120003699FECF85B10895811104C01BBC19BC5E
:1001300018BC0895815090E0FC01E25EFF4FE4910D
:10014000EBBDFC01EA5BFF4FE491E9BDFC01E25924
:10015000FF4F849188BD08950F931F93CF93C82FAD
:100160008B01CC2369F08AE0DFDFC801BFDF1BBC55
:1001700019BC18BCC801BADFC801B8DFC150F1CF43
:10018000CF911F910F910895CF93DF93D82F64E102
:1001900070E08AE0E1DF84EF91E0A8DF8D2F64E674
:1001A00053D0CAE06C2F50D0892F68EC70E0D4DFB8
:1001B000ADDF8D2F6C2F48D0D92F46D0892F68EC1A
:1001C00070E0CADFA3DF68EC70E08D2FC5DF9EDF33
:1001D00064E170E08AE0C0DF84EF91E0DF91CF91CD
:1001E00085CF83EA87B986EC86B93699FECF369AF1
:1001F0003699FECF85B18FE384BBBB9AC39AB99A77
:10020000B89ABC9A81E08ABD83BF9AB590629ABDC4
:100210009AB590689ABD9FEF9DBD80BF80E68CBD6A
:1002200097B328B3892F90E0809590958B7F822B90
:1002300088BB85B7806285BF78946BDF8CE291E0E4
:1002400055DF6DDFA1DFFACF991B79E004C0991F5C
:10025000961708F0961B881F7A95C9F78095089520
:04026000F894FFCF40
:00000001FF
